:020000000C945E
:100002006A000C9400000C9400000C9400000C9404
:1000120000000C9400000C9400000C9400000C945E
:1000220000000C9400000C9400000C9400000C944E
:1000320000000C9400000C9400000C9400000C943E
:10004200CC000C9400000C9499000C9400000C94C9
:1000520000000C9400000C9400000C9400000C941E
:1000620000000C9400001027E80364000A0001005D
:100072000010000110000100000000000A00000052
:10008200000000000000000000000000000000006E
:10009200000000000000000000000000000000005E
:1000A200000000000000000000000000000A0A0A30
:1000B2000A0A0A0A0A0A0A0A0A0A0A0A0A000200BA
:1000C20002007A00020004007C00010009037E00A5
:1000D2000000F894EE27EFBBF1E0F5BFE5BF8DE03D
:1000E200A2E0BB27ED938A95E9F780E098E0A0E0D3
:1000F200B1E0ED930197E9F7E0ECF0E0859195919D
:10010200009761F0A591B59105901590BF01F0019E
:1001120005900D920197E1F7FB01F0CFE8E0EEBB0D
:10012200EFEFEDBFE8E0EEBFC0E0D3E00C944C038C
:10013200AA93EA93FA93EFB7EA931A930A93109168
:10014200C0000091C600E12FEC71E9F4E091D60302
:10015200EF5FE093D603E150F0E0E354FC4F0083FD
:10016200A091D603A93119F4E0E0E093D603A0915F
:10017200D803AF5FA093D803A93129F4E0E0E0935C
:10018200D803689435F809911991E991EFBFF99173
:10019200E991A99118950A921A926A937A938A938D
:1001A2009A93AA93BA93EA93FA93EFB7EA93E091F8
:1001B2003103F09132033196E0933103F09332032D
:1001C2000E94351BE1E5F1E00E94BB240E2E0E9445
:1001D200351BE3EAF2E00E94BB24E02909F4C1C125
:1001E200A0912F03B0913003E4E1F0E00E94CD240E
:1001F2000E2EE0910603F0E074970E94C1240E22B5
:10020200A0911E03EEE00E94B124E02121F0E091D2
:100212001E03EF5F03C025FC03C0E0E0E0931E0372
:10022200A0911E03AE3011F4689425F8E0912F03DB
:10023200E0930603A0911F03A13029F4F79B02C0AB
:10024200F79801C0F79AE1E02E260E943A1B0E941D
:10025200431BE093A503F093A6036093A703709357
:10026200A8030E944A1BA9E8B3E00E944F1B0E9408
:10027200561BA5EBB3E00E944F1B0E945B1B0E9422
:10028200641B0E94E723E0938903F0938A0360933F
:100292008B0370938C03A091B503B091B603809148
:1002A200B7039091B803E0E0F0E060E772E40E94E7
:1002B200E723E093B503F093B6036093B70370931B
:1002C200B8030E94691B0E946E1B0E2E0E94731BB4
:1002D2000E946E1BE02161F1E091B503F091B6033B
:1002E2006091B7037091B8030E945B1B0E94E723E1
:1002F200E093B103F093B2036093B3037093B4033A
:100302000E94781BA5E4B3E00E94811BA091B10377
:10031200B091B2038091B3039091B4030E94431B46
:10032200E0939103F0939203609393037093940389
:100332000E94861BE0E0F0E06AE774E40E948F1BF3
:100342000E94941B0E944923E0939903F0939A031D
:1003520060939B0370939C030E949D1B0E94A21BAF
:100362000E94B31BAFE5B3E00E94B81B0E94BD1B05
:100372000E94861B0E940F230E948F1BE093A903F9
:10038200F093AA036093AB037093AC03A091B903FB
:10039200B091BA038091BB039091BC030E944923A0
:1003A200E093B903F093BA036093BB037093BC0369
:1003B2000E949D1BE5E20E94C61BA1E6B3E00E94DB
:1003C200B81B0E943A1B0E940526DCF40E94D61B31
:1003D200A0E0B0E080E89FE30E94E723A091A90398
:1003E200B091AA038091AB039091AC030E94992330
:1003F200E093A103F093A2036093A3037093A40379
:1004020009C0E0E0E093A103E093A203E093A30319
:10041200E093A4030E94DF1BA4E2B3E00E94D62271
:10042200EC930E94D61B0E94E81B0E9449230E9463
:10043200F11BE0918903F0918A0360918B03709123
:100442008C030E94FA1B0E942C2468F5E091910310
:10045200F091920360919303709194030E94FA1BAE
:100462000E944923E0938D03F0938E0360938F03E0
:10047200709390030E94FA1B0E94031C0E94422365
:10048200DF01CB010E94781B0E94E723A0E0B0E0CD
:1004920081E695E40E949923ABE5B3E00E94B81B84
:1004A200689424F802C0E0E12E260E94D61B0E9426
:1004B2000C1C0E944923E0939503F09396036093EA
:1004C2009703709398030E940C1CE0E0F0E060E850
:1004D2007FE30E942C2409F008F416C0E0939503F0
:1004E200E0939603E0939703E09398030E94151C10
:1004F200EF5FFF4F6F4F7F4F0E941E1C0E94151C23
:10050200AEE2B0E00E94DA250E94271CA034E2E4A9
:10051200BE07EFE08E07E0E09E0778F0E0E0E093B0
:100522005103E0935203E0935303E0935403AEE28A
:10053200B0E00E94301C0E94DA250E94E81B0E9453
:10054200641B0E949923A3E3B3E00E94811BA09144
:100552001C03AC3308F4F298A0911C03AC3309F4E9
:10056200F29A0E94351BA33AE2E0BE0709F06AC084
:10057200A0911B030E94351C0E943A1C0E94301C51
:100582000E94D3240E94431CE02191F0E0911C03BD
:10059200EF5FE0931C03E0911B03F0E03296A09121
:1005A2001C03B0E0EA17FB0719F4ECE3E0931C0329
:1005B200E0E0E0933103E0933203C3940E944A1CCB
:1005C200E8E5F2E00E94C7240E2E0E944F1CE021B3
:1005D200E9F0E0914903F0914A033196E09349032F
:1005E200F0934A030E944A1C0E94541CEA1BFB0B14
:1005F200E0934F03F09350030E943A1C0E94052699
:100602002CF4E0E0E0934903E0934A03ECE3EC15B9
:10061200C9F4CC24E0910003EF5FE0930003A091C2
:100622000003AC3379F4E0E0E0930003E0910103CE
:10063200EF5FE0930103A0910103A43119F4E0E01C
:10064200E0930103E991EFBFF991E991B991A99181
:100652009991899179916991199009901895AA9324
:10066200E881E066E0937C0085E28A95F1F7E0910B
:100672007A00E064E0937A00E0917A00E071E1F3BD
:10068200E0917A00E061E0937A00E0917800F091E5
:10069200790021960895EF9722978FE3A2E0B0E0C8
:1006A200E0E8F0E00E941A26FF2401E021E0E0E801
:1006B200E0936100E0E0E0936100EFE0E4B9E1E0A3
:1006C200E5B9E0E0E7B9E4E0E8B9EAEFEAB9E7EE74
:1006D200EBB9E0E0E4BDE3E0E5BDE0E0E6BDE7BDA7
:1006E200E8BDE1EAE0938000E2E0E0938100E0E02F
:1006F200E0938500E0938400E0938700E093860016
:10070200E0938900E0938800E0938B00E0938A00F5
:10071200E093B600E1EAE093B000E2E0E093B100DA
:10072200E0E0E093B200E093B300E093B400E1E0D4
:10073200E0936E00E0E0E0936F00E0937000E093DE
:100742006900EDBBE0936800E093C000E8E9E09344
:10075200C100E6E0E093C200E0E0E093C500E7E418
:10076200E093C400E0E8E0BFE0E0E0937F00E093C4
:100772007E00E0E6E0937C00E7E2E0937A00E0E0CE
:10078200E0937B00ECBDE093BC0078940E94591C7E
:100792000E94611C0E946E1C0E947B1CEAE09E1655
:1007A20030F4A0E2B0E0E0E0F0E00E94E225EAE00E
:1007B2008E1640F4A6E2B0E0E0E0F0E00E94E2250E
:1007C200689426F8EAE0AE1618F4689430F827F830
:1007D200689433F80E94851C0E948C1C0E94931C12
:1007E200E8ECF0E0E0935503F0935603E1E1E09387
:1007F2001003A0E0B0E00E94CE25E0931103A1E037
:10080200B0E00E94CE25E0931203A2E0B0E00E9485
:10081200CE25E0931303A3E0B0E00E94CE25E0933F
:100822001503A4E0B0E00E94CE25EF8BA5E0B0E076
:100832000E94CE25E88FA6E0B0E00E94CE25E98F87
:10084200A7E0B0E00E94CE25E0931603A8E0B0E056
:100852000E94CE25E0931703A9E0B0E00E94CE25C6
:10086200E0931803F798F198AAE0B0E00E94CE2531
:10087200E0931B03AEE1B0E00E94CA250E949A1CDD
:10088200A4E1B0E00E94CE25EB8BA5E1B0E00E948E
:10089200CE25EC8BA6E1B0E00E94CE25ED8BABE03D
:1008A200B0E00E94CE25EF87ACE0B0E00E94CE25FA
:1008B200E88BADE0B0E00E94CE25E98BA2E2B0E089
:1008C2000E94CA25ED83FE83AEE0B0E00E94CE25F1
:1008D200E0932003AFE0B0E00E94CE25E093220334
:1008E200A0E1B0E00E94CE25E0932103AEE2B0E0A9
:1008F2000E94C6250E941E1CA0E2B0E00E94CA25EA
:10090200A5E8B3E00E949F1C0E94031CA3E3B3E08E
:100912000E94811B0E94E81B0E94641B0E94E72325
:100922000E94F11BA1E1B0E00E94CE253E2FA4E27D
:10093200B0E00E94CA25E987FA87A2E1B0E00E94EE
:10094200CE25EB8FA3E1B0E00E94CE25EA8FA6E28E
:10095200B0E00E94CA25A9E9B3E00E949F1CA8E268
:10096200B0E00E94CA250E94A61CACE2B0E00E9440
:10097200CA250E94AB1CA7E1B0E00E94CE250E94CE
:10098200152623F8AAE2B0E00E94CA250E94B01CF4
:10099200A8E1B0E00E94CE25E0930803A9E1B0E00F
:1009A2000E94CE25E0930A03AAE1B0E00E94CE2580
:1009B200E0930B03ABE1B0E00E94CE25E0930C0381
:1009C200ACE1B0E00E94CE25E0930D03ADE1B0E0D2
:1009D2000E94CE25E0930E03A0910303A43128F4D4
:1009E200E0910303EF5FE0930303A0910303A431BB
:1009F200A1F4E0E0E0932603E0932703EBE0F0E0CC
:100A0200E0934D03F0934E03E8EBE0932803E0E01C
:100A1200E093D603EAE0E0930303A091D603AB3060
:100A2200C1F4E091C003E0932603E091C103E09397
:100A32002703E091C203F0E0E0934D03F0934E03ED
:100A4200E091C303E0932803E0E0E093D603E09350
:100A52000303A091D603AC30C0F0E0E0E093BD0305
:100A6200E093BE03E093BF03E093C003E093C103AE
:100A72000E94851CE0E0E093C403E093C503E09389
:100A8200C603E093C703E093D603E8EC5E1630F4A6
:100A92005394E4E1E51511F4E1E04E2E0E94591C55
:100AA200A0E00E94B51C3B9798F1A0E00E94BA1CFE
:100AB200662777270E94C11C0E94BD1BA8EEB3E0E7
:100AC20080E090E00E941E25DF01CB010E94CA1C3B
:100AD200662777270E9460250E94C11CE0910903C6
:100AE200EF5FE0930903E0910803A0910903AE17B9
:100AF20068F00E94BD1BE0937503F0937603609348
:100B0200770370937803E0E0E0930903E894F3F845
:100B12000E94CF1C0E94611CA2E00E94BA1CDF014D
:100B2200E5E0F0E00E942325BE2E0E94CF1C0E9429
:100B32006E1CA7E00E94B51C0E94D61C0E94CF1C0E
:100B4200A5E00E94B51C1E2F0E94CF1CA0E00E94AF
:100B5200B51CDE2E0E94CF1C0E947B1CE7EAE093AC
:100B62007A00A6E00E94B51CED87E7E2E0937A00E6
:100B7200E1E0E51591F50E94DB1CE2E3F0E00E9462
:100B8200CD240E2E0E94E01C0E94C724E02111F009
:100B9200E5E0EC87A12FE2E30E94B6240E2EEAEFF5
:100BA2000E94B124E02111F0E6E0EC870E94E01CF3
:100BB2000E94CD240E2E0E94E41CE02911F0E7E0F1
:100BC200EC87A12FEAEF0E94B6240E2EEEE10E94DE
:100BD200B124E02911F0E8E0EC870E94E01C0E94B9
:100BE200CD240E94EA1C39F0E1E0EC87E8E2F0E073
:100BF2000E94D61C07C00E94E41C0E94EA1C11F04D
:100C0200E2E0EC87A12FEAEF0E94B6240E94EA1CE0
:100C120011F0E3E008C0A12FEEE10E94B1240E948E
:100C2200EA1C19F0E4E0EC871CE3AC850E94F61C98
:100C3200AC85E7E00E9498240E2AE1E00E94982405
:100C42000E2AE2E00E949824E02929F0E12FF0E048
:100C52000E94D61C18E2AC850E94FB1CAC85E8E021
:100C62000E949824E02909F018E20E94001D0E94C7
:100C7200061D0E94B124E021D1F06894F3F80130FE
:100C820021F4F398F49A02E012C0023059F4F49875
:100C9200F59AA98DA13010F003E003C0F598F39AFC
:100CA20001E005C0033019F4F598F39A01E00E94BF
:100CB200DB1CD39708F457C00E94101D0E94151D1B
:100CC200E02F0E941C1D20F0E8ECF0E00E94D61CF0
:100CD200E02F0E942C1D0E943C1DAC91A13008F413
:100CE20041C00E94431D0E944C1D0E9410264CF4DC
:100CF2000E943C1D0E94581D0E9458240E94631DA0
:100D020023C00E946C1D0E946E1DEF930E946C1DF9
:100D12000E94771DAF91EA2379F00E943C1D0E9448
:100D2200581D0E945D24A0936503B09366038093CF
:100D320067039093680308C00E946C1D0E94801D87
:100D42001CF00E948A1D0EC0A0916503B09166033B
:100D520080916703909168030E94991D0E9460250B
:100D62000E94D61C04C00E949E1D0E948A1D0E94E1
:100D7200A41D0E94AA1D0E220E94AF1DE02139F07F
:100D8200E0912D03E0931D036894F0F821F80E948E
:100D9200101D309721F4E0E0E0931E0306C0A091FD
:100DA2001E03A23010F4E89425F80E94101DE0936F
:100DB2002F03F09330030E94101D309719F4E8942A
:100DC20021F815C0A0E021FCA1E0E0E00E949824F7
:100DD2000E2EA0911D03E0E00E94B624E02139F01E
:100DE200E0E0E0931D030E949E1DE89422F8E0914A
:100DF20005030E94DB1CF0E0AE17BF0720F0E09174
:100E02002D03E0930503E0910503F0E035970E947E
:100E1200DB1CAE17BF0770F4E0912D03E0930503CE
:100E220025FE08C0E2E0E0932303E89425F8E0E021
:100E3200E0931E03A0911D03A13080F0689422F874
:100E42000E94101DA0911D03B0E0AE17BF0728F04D
:100E5200E0911D03F0E00E94D61C02C0E89422F843
:100E62000E94B61D0E94B91D0E94E3240E22A09189
:100E720020030E94C01D1E2E0E94B61D0E94B91D95
:100E82000E94DB240E22A09121030E94C01D1E2A73
:100E92000E94B61DA12FE2E30E94B624E021E129BF
:100EA20079F00E949E1DA0912303A13021F4EAE073
:100EB200F0E00E94D61CE0912303E150E09323036B
:100EC2000E94C51D0E22A0E031FCA1E00E94C01DBF
:100ED20031F0689431F80E94101D0E94DB1D0E94BF
:100EE200C51DE02161F10E94E01D0E94E81DA4F0F1
:100EF200A0917103B0917203ED81FE81EA1BFB0B9D
:100F0200A3E0B0E00E9419250E94F01DAE1BBF0BAA
:100F1200A0935703B09358030E94E01D0E94052638
:100F22002CF40E94F51D32970E94DB1DA0915803FC
:100F3200AA232AF4E0E0E0935703E09358030E94C7
:100F4200FA1D0E940B2674F50E94FA1D0E945D2470
:100F52000E94E81D74F0AD81BE81E0917103F091B1
:100F62007203EA1BFB0B0E94F01DEA0FFB1F0E949B
:100F7200DB1D0E94FA1D0E945D24A230E0E0BE0744
:100F8200E0E08E07E0E09E072CF00E94F51D31960E
:100F92000E94DB1D0E94F01DA93CE0E0BE0714F098
:100FA2000E948C1C0E94F51D0E94DB1CAE17BF071D
:100FB20010F4E89431F80E94F51D0E94DB1CEA1738
:100FC200FB0720F40E94F51D0E94D61C0E94071EFA
:100FD2000E9452240E2EA0E032FCA1E00E94C01D0D
:100FE20041F0689432F80E94161EE0935903F09380
:100FF2005A030E94071E0E942C2409F008F435C0EF
:101002000E941B1EDF01CB01E0E0F0E060E070E433
:101012000E942C2409F008F410C00E941B1EDF015C
:10102200CB01E985FA850E942A1E0E94311E0E9488
:10103200361EA9E5B3E00E94B81B0E941B1E0E9447
:10104200FB2554F4EB8DF0E00E94311EAE1BBF0B6A
:10105200A0935903B0935A03A0915A03AA232AF4E6
:10106200E0E0E0935903E0935A030E94071E0E94B6
:101072002C24D0F50E943B1EDF01CB01E0E0F0E022
:1010820060E470E40E942C2409F008F416C00E9467
:101092003B1EA0E0B0E080EA90E40E949923DF01C9
:1010A200CB010E94461E0E948E240E940F230E94A2
:1010B2004923A9E5B3E00E94B81B0E943B1E0E948F
:1010C200FB2554F4EA8DF0E00E94311EEA0FFB1F6B
:1010D200E0935903F0935A030E94311EA13DE7E0C9
:1010E200BE0714F00E94931C0E94161EDF010E948C
:1010F200461EAE17BF0710F4E89432F80E94161E7F
:10110200DF010E94461EEA17FB0720F40E94311EEF
:101112000E944B1E0E94501E0E94E3240E2EA0E04D
:1011220034FCA1E00E94C01D31F0689434F80E94A2
:10113200161E0E94571E0E94501E0E940B265CF52E
:101142000E945C1E0E94E81D9CF0E0911203F0E0F8
:10115200A0916D03B0916E03AE1BBF0BE3E0F0E014
:101162000E94651EAE1BBF0BA0936303B093640382
:101172000E945C1E0E9405262CF40E946C1E32976F
:101182000E94571EA0916403AA232AF4E0E0E09390
:101192006303E09364030E94501E0E9410268CF5A4
:1011A2000E94711EA430E0E0BE07E0E08E07E0E09E
:1011B2009E078CF0A0911203BB27E0916D03F09182
:1011C2006E03AE1BBF0BE2E0F0E00E94651EEA0F69
:1011D200FB1F0E94571E0E94711E0E9405262CF4BE
:1011E2000E946C1E32960E94571EA0916303B0911A
:1011F2006403A13DE7E0BE0724F0E0EDF7E00E94C2
:10120200571E0E94161EDF010E946C1EAE17BF07FA
:1012120010F4E89434F80E94161EDF010E946C1E3E
:10122200EA17FB0730F4A0916303B09164030E94B4
:101232004B1E1333D8F0A0911D03A13018F0E2E049
:10124200E0932303E0E0E0931D03E12FF0E0F29747
:101252000E948E240E940F23A6EFB8E28CE99FE33E
:101262000E9499230E94D6221E2F01C010E00E94E4
:10127200101DEB83FC83AB2DE4E60E94B1240E2EFD
:10128200A0E0F099A1E0E1E00E9498240E94431CB2
:101292000E22AA81EDE50E949D24E0211E2E0E94CD
:1012A200541C0E944A1C0E94BB240E94811E0E9460
:1012B2004F1CE021E129C9F0E0913303F09134039E
:1012C200A0E2B0E00E94E2250E94891E0E94E51E73
:1012D2000E944E1FA4E6B0E00E949F225F98A8EEF3
:1012E200B3E00E949F220C94281BAA2D0E94691F22
:1012F2000E94AA1DE02131F0E894F2F827F8E0E01C
:10130200E0932C030E946E1F0E94AA1DE02171F03F
:10131200E0912C03EF5FE0932C03A0912C03AA3001
:1013220029F4E0E0E0932C03E0931F030E946E1F78
:101332000E947B1F0E94AA1DE02171F06894F2F8BE
:10134200E0911F03EF5FE0931F03A0911F03A330FF
:1013520019F4E1E0E0931F03E0911F03E03029F468
:10136200E0E0E093B400F7980FC0A0911F03A13012
:1013720019F4E091180306C0A0911F03A23021F4D2
:10138200F79AEFEFE093B4000E94DB1C0E946E1B01
:101392000E2EA12FE0E00E94B6240E22A0E022FC35
:1013A200A1E00E94C01D01F1E0910403EF5FE09310
:1013B2000403A0910403E5E00E94B6240E2EE4E1AA
:1013C2000E94B124E02141F0E0910403E170AFEF0B
:1013D200EA02F001E093B400A0910403A03118F0F6
:1013E200E0E0E093040326C0A0E030FCA1E0E1E0ED
:1013F2000E9498240E2EA0911F030E94C01DD1F0BE
:10140200E0912B03EF5FE0932B03A0912B03A1301C
:1014120019F4EFEFE093B400A0912B03A33019F479
:10142200E0E0E093B400A0912B03A43019F4E0E0D3
:10143200E0932B03E0911703E093B300EAE0E81591
:1014420018F4E894F1F826F80E94831FA0E026FC25
:10145200A1E00E94891FA0E0F1FCA1E00E94891F87
:101462000E94AA1DE02139F16894F1F8E0910F037E
:10147200EF5FE0930F03E0E0EB87AB85A53088F4E4
:101482000E948E1FA081A13018F0E5E0EB8705C015
:10149200E0910F03EF5FE0930F03EB85EF5FEB87C4
:1014A200ECCFA0910F03A53018F0E0E0E0930F031A
:1014B2000E948E1F20810E94831FA0911A03EFEFCA
:1014C2000E94B124E02121F0E0911A03EF5F03C0F2
:1014D200E894F1F8E0E0E0931A03A0911A03A43132
:1014E200E1F4AA81E0E00E94AC240E2E0E94AA1D23
:1014F200E02119F0EA81E150EA83233610F423E671
:101502000CC021E0E0E0E0930F030E94891E0E94DC
:10151200E51E0E944E1FE1E04E2E0E94831FA0E0B6
:10152200F1FCA1E00E94891FAA81E4E60E94A7249F
:101532000E94941F51F06894F1F8EA81EF5FEA8308
:10154200AA81A43611F4E0E0EA83EAE0E91510F496
:10155200E894F0F80E94A41D0E94AF1D0E22AA81F9
:10156200E0E00E94A2240E94941F51F06894F0F8D7
:10157200EA81E150EA83AA81AF3F11F4E3E6EA830C
:101582000E94001D0E949B1FC1F00E94A11FA9F48E
:10159200A0912903A43119F4E7E0E0932903E0E0E4
:1015A200E0932A03E894F3F8A0912903A33028F0EA
:1015B200E0912903E150E0932903AA2DEAE00E9479
:1015C200B1240E2E0E949B1FC1F00E94A11FA9F4FC
:1015D200A0912903A43119F4E7E0E0932903E0E0A4
:1015E200E0932A03E894F2F8A0912903A33028F0AB
:1015F200E0912903E150E0932903AA2D0E94691F7B
:10160200AD2DEAE00E94B624E02131F0E0E0E09363
:101612002A03E4E1E0932903EAE0ED1510F4E894EB
:10162200F3F80E94001D0E94061D0E949824E021EA
:1016320009F4D1C16894F3F8AA81A13049F4A091C8
:101642001103A13028F4E0911103EF5FE09311033D
:10165200AA81A23049F4A0911203A23328F4E091A6
:101662001203EB5FE0931203AA81A33049F4A09125
:101672001303A43628F4E0911303EF5FE0931303FE
:10168200AA81A43049F4A0911503A83228F4E0916C
:101692001503EF5FE0931503AA81A53031F4AF89FA
:1016A200A43618F4EF89EF5FEF8BAA81A63031F4EC
:1016B200A88DA43618F4E88DEF5FE88FAA81A730D1
:1016C20031F4A98DA43618F4E98DEF5FE98FAA8170
:1016D200A83049F4A0911603AF3F28F4E091160315
:1016E200EF5FE0931603AA81AD3069F4A091350350
:1016F200B0913603A433E8E0BE0728F40E94CA1C66
:1017020031960E949A1CAA81AE3031F4AB89A4367C
:1017120018F4EB89EB5FEB8BAA81AF3031F4AC8923
:10172200A43618F4EC89EB5FEC8BAA81A03131F47A
:10173200AD89A43618F4ED89EB5FED8BAA81A13156
:1017420031F4AF85A83C18F4EF85EB5FEF87AA81EF
:10175200A23131F4A889A83C18F4E889EB5FE88B40
:10176200AA81A33131F4A989A83C18F4E989EB5F75
:10177200E98BAA81A43169F4A0914703B09148038F
:10178200A835E2E0BE0728F40E94541C7E960E940F
:10179200B01CAA81A53159F4AD81BE81A33AE1E022
:1017A200BE0728F4ED81FE813196ED83FE83AA8186
:1017B200A63149F4A0912003A13028F4E09120033E
:1017C200EF5FE0932003AA81A73149F4A09122039D
:1017D200A23328F4E0912203EF5FE0932203AA816F
:1017E200A83149F4A0912103A13028F4E09121030A
:1017F200EF5FE0932103AA81A93119F43F3008F485
:101802003F5FAA81AA3159F40E94AC1FAC3BE2E0CF
:10181200BE0728F40E94B11F31960E94A61CAA811D
:10182200AB3159F40E949D1BA73EE3E0BE0728F4AA
:101832000E94B61F31960E94AB1CAA81AC3161F4A2
:10184200A0E023FCA1E0A13038F4E0E023FCE1E0D9
:10185200EF5F0E94152623F8AA81AD3169F40E9438
:10186200691BAE3DE3E0BE0738F40E944A1B3A967C
:10187200E0933D03F0933E03AA81AE3169F40E94E6
:10188200731BA835E2E0BE0738F40E94561B3A9655
:10189200E0934B03F0934C03AA81AF3149F4A0913A
:1018A2000803AA3028F4E0910803EF5FE0930803ED
:1018B200AA81A03249F4A0910A03A93028F4E09148
:1018C2000A03EF5FE0930A03AA81A13249F4A091CF
:1018D2000B03A93028F4E0910B03EF5FE0930B03B5
:1018E200AA81A23249F4A0910C03A93028F4E09114
:1018F2000C03EF5FE0930C03AA81A33249F4A09199
:101902000D03A93028F4E0910D03EF5FE0930D037E
:10191200AA81A43249F4A0910E03A93028F4E091DF
:101922000E03EF5FE0930E03AA81AC3549F4A09158
:101932000703AA3F28F4E0910703E65FE093070359
:10194200AA81AD3531F4AC8DA73018F4EC8DEF5F80
:10195200EC8FAA81AE3549F4A985BA851A9728F485
:10196200E985FA853196E987FA87AA81AF3531F49C
:10197200AB8DAA3018F4EB8DEF5FEB8FAA81A03606
:1019820031F4AA8DAA3018F4EA8DEF5FEA8FAA81AA
:10199200A13649F4A0911B03AC3328F4E0911B0358
:1019A200EF5FE0931B03AA81A23649F4A0911803CA
:1019B200AA3F28F4E0911803E65FE0931803AA8196
:1019C200A33649F4A0911703AA3F28F4E091170324
:1019D200E65FE0931703EAE0EA1510F4E894F2F800
:1019E200AA2DEAE00E94B1240E2E0E947B1F0E94C3
:1019F2009B1F09F4CEC16894F2F8AA81A13049F480
:101A0200A0911103A13028F0E0911103E150E0937D
:101A12001103AA81A23049F4A0911203AB3028F03D
:101A2200E0911203E550E0931203AA81A33049F436
:101A3200A0911303AD3328F0E0911303E150E0933A
:101A42001303AA81A43049F4A0911503A53128F00B
:101A5200E0911503E150E0931503AA81A53031F41A
:101A6200AF89A13018F0EF89E150EF8BAA81A6303F
:101A720031F4A88DA13018F0E88DE150E88FAA81E9
:101A8200A73031F4A98DA13018F0E98DE150E98F2A
:101A9200AA81A83049F4A0911603A13028F0E09160
:101AA2001603E150E0931603AA81AD3069F4A091C8
:101AB2003503B0913603AD36E7E0BE0728F00E9449
:101AC200CA1C31970E949A1CAA81AE3031F4AB89AC
:101AD200A63018F0EB89E550EB8BAA81AF3031F4D8
:101AE200AC89A63018F0EC89E550EC8BAA81A031C4
:101AF20031F4AD89A63018F0ED89E550ED8BAA815D
:101B0200A13131F4AF85A13018F0EF85E550EF87B0
:101B1200AA81A23131F4A889A13018F0E889E550F0
:101B2200E88BAA81A33131F4A989A13018F0E9899F
:101B3200E550E98BAA81A43161F4A0914703B091E9
:101B420048030E94012628F40E94541C7E970E949A
:101B5200B01CAA81A53159F4AD81BE81A332E1E066
:101B6200BE0728F0ED81FE813197ED83FE83AA81C5
:101B7200A63149F4A0912003A13028F0E09120037E
:101B8200E150E0932003AA81A73149F4A0912203F6
:101B9200A23028F0E0912203E150E0932203AA81CF
:101BA200A83149F4A0912103A13028F0E09121034A
:101BB200E150E0932103AA81A93119F4323008F0EF
:101BC2003150AA81AA3159F40E94AC1FA935E2E032
:101BD200BE0728F00E94B11F31970E94A61CAA815D
:101BE200AB3149F40E949D1B1B9728F00E94B61F3F
:101BF20031970E94AB1CAA81AC3179F4A0E023FC9E
:101C0200A1E0A13050F0A0E023FCA1E0E1E00E94BD
:101C1200C225EA1B0E94152623F8AA81AD3161F480
:101C22000E94691B0E94012638F40E944A1B3197C8
:101C3200E0933D03F0933E03AA81AE3161F40E942A
:101C4200731B0E94012638F40E94561B3197E093C1
:101C52004B03F0934C03AA81AF3149F4A0910803DE
:101C6200A23028F0E0910803E150E0930803AA8132
:101C7200A03249F4A0910A03A23028F0E0910A03AD
:101C8200E150E0930A03AA81A13249F4A0910B0327
:101C9200A13028F0E0910B03E150E0930B03AA81FD
:101CA200A23249F4A0910C03A13028F0E0910C0378
:101CB200E150E0930C03AA81A33249F4A0910D03F1
:101CC200A13028F0E0910D03E150E0930D03AA81C9
:101CD200A43249F4A0910E03A13028F0E0910E0342
:101CE200E150E0930E03AA81AC3539F4A0910703C9
:101CF200A13018F0E0E0E0930703AA81AD3531F49A
:101D0200AC8DA13018F0EC8DE150EC8FAA81AE358C
:101D120051F4A985BA850E94012628F4E985FA853D
:101D22003197E987FA87AA81AF3531F4AB8DA130BB
:101D320018F0EB8DE150EB8FAA81A03631F4AA8D19
:101D4200A13018F0EA8DE150EA8FAA81A13649F458
:101D5200A0911B03A13028F0E0911B03E150E09316
:101D62001B03AA81A23649F4A0911803AB3028F0D4
:101D7200E0911803EA50E0931803AA81A33649F4CC
:101D8200A0911703A13028F0E0911703EA50E093E5
:101D9200170323FC26C0E0912703ADEAB3E0FF2737
:101DA200662777270E940F230E94AF25A091AD03DB
:101DB200B091AE038091AF039091B0030E940526CB
:101DC2003CF40E94BB1F0E94C41F0E94CB1F09C08B
:101DD200E0E0E0939D03E0939E03E0939F03E09392
:101DE200A00323FE0BC0AD850E94D41FADEAB3E071
:101DF2000E949F1C0E94BB1F0E94CB1F0E94BB1F00
:101E0200A5E2B3E00E94D622EC93F0914D03E0E00C
:101E1200DF01E0912803F0E0EA0FFB1FADE7B3E03A
:101E22000E944F1B0E94DA1FA0E0B0E080E192E422
:101E32000E94E7237F936F93FF93EF930E94AC1F5F
:101E42000E94E31FAF91BF918F919F910E942A1E22
:101E5200E0937D03F0937E0360937F03709380038E
:101E62000E94E81FE0E0F0E060E87FE30E94522475
:101E72000E2E0E94E81FE0E0F0E068E472E40E94A7
:101E82004C24E021F9F00E94DA1F0E94C41FADE643
:101E9200B3E00E94D8220E94AF250E94DA1FE0938D
:101EA2008103F093820360938303709384030E94FF
:101EB200E81F0E94641B0E949923A7E3B3E00E94DB
:101EC200811B15C0E0E0E0936D03E0936E03E093A5
:101ED2006F03E0937003E0938103E0938203E09346
:101EE2008303E0938403E0933703E0933803A091E4
:101EF200A103B091A2038091A3039091A4030E9435
:101F0200301C0E945224EF930E94F11F0E9452241F
:101F1200AF91EA23C9F10E94941BE0E0F0E068EC83
:101F220072E40E94E7230E949D1B882799270E9442
:101F3200B6250E94B31B0E94F31FA0917903B091B2
:101F42007A0380917B0390917C03E0E0F0E064E10E
:101F520072E40E949923DF01CB010E94DF1B0E94E1
:101F6200E723A0E0B0E080E291E40E9499230E947E
:101F7200F31FE0917903F0917A0360917B037091F2
:101F82007C03DE010E94B81B0E94A41DA0911903CC
:101F9200EDEF0E94B1240E220E94AA1DE02129F039
:101FA200E0911903EF5FE0931903A92D0E94691FC5
:101FB200A0911903EFEF0E94B1240E220E94AA1DE4
:101FC200E02129F0E894F0F8E0E0E0931903A09111
:101FD2001903EEE10E9498240E2E0E94AA1DE02110
:101FE20019F0E1E0E0931C03E0911B03E03019F4E7
:101FF200E0E0E0931C030E943A1C0E94301C0E9405
:10200200E3240E94811EA0911C03E0E00E94B624FA
:10201200E02119F0E1E0E0931C03A0911C03AC3332
:1020220009F41FEFA0910703A13028F0E091070304
:10203200F0E00E94D61C4420C9F4E02FF0E0349670
:102042000E94DB1CAE0FBF1FE12F0E94FC1FA4E009
:102052000E942B1BA02F0E940620A0912D030E94FC
:102062002B1BA12F0E942B1B0E940B20E1E0E415E9
:1020720009F057C04424A09113030E941420E09356
:102082001403F0E0BC96DF01E0911003F0E0AE0F24
:10209200BF1FE0911103F0E0AE0FBF1FE0911203EA
:1020A200F0E0AE0FBF1FE0911503F0E0AE0FBF1FCF
:1020B200EF89F0E0AE0FBF1FE88DF0E0AE0FBF1F5B
:1020C200E98DF0E0AE0FBF1FE09116030E94FC1FE6
:1020D200ACE20E942B1BA09110030E942B1BA0912B
:1020E20011030E942B1BA09112030E942B1BA09193
:1020F20014030E942B1BA09115030E942B1BAF8976
:102102000E942B1BA88D0E942B1BA98D0E942B1BAA
:10211200A09116030E940620A0E00E9406200E94C1
:102122000B20233608F086C30E948E1F2081A0E078
:10213200F799A1E0EA2FE295E07F0E2EA0E0F39955
:10214200A1E0EA2FEE0FEE0F0E0EA0E0F499A1E04F
:10215200EA2FEE0FA02DAE0FE0E0F599E1E0EA0FD5
:10216200ED8FEAE0EAABEBABECABEDABEEABEFAB9A
:10217200E8AF0E941A20EAE0ECAFEDAFEEAFEFAFAE
:10218200DE01A05CBF4FEC930E941F20AA34E1E065
:10219200BE07E0E08E07E0E09E071CF4E1E0E0937A
:1021A20002030E941F20E9E4F1E060E070E00E9477
:1021B2002820EEE5F1E060E070E00E94DB24E021FF
:1021C20019F0E3E0E09302030E941F20EDE5F1E045
:1021D20060E070E00E942820E8E6F1E060E070E054
:1021E2000E94DB24E02119F0E7E0E09302030E9461
:1021F2001F20E7E6F1E060E070E00E942820ECE7B3
:10220200F1E060E070E00E94DB24E02119F0EFE0F1
:10221200E09302030E941F20AC37E1E0BE07E0E03A
:102222008E07E0E09E071CF0EFE1E09302030E94BC
:102232003A1C0E942C202CF00E9434200E943A204A
:10224200ECAB0E9434200E947A25EDABA0912503CD
:10225200AA3028F00E94D41F0E944520EAAB0E94B7
:102262004B20EBAB0E941F200E9453200E943A2079
:10227200EEAB0E9458200E943A20EFAB0E945820F9
:102282000E947A25E8AF213011F50E945E200E945B
:102292007520E7550E9484200E948E20A436E0E03B
:1022A200BE0710F00E9493200E948E200E94E31F1E
:1022B2000E949F200E94A5200E94AB2010F0E2E025
:1022C200E9AF0E94B6200E9445200E94C120223020
:1022D20009F065C00E945E200E94CB20E75B0E944D
:1022E20084200E94271CA03AE6E8BE07E1E08E07A0
:1022F200E0E09E0748F00E94271CE0EAF6E861E071
:1023020070E00E94D320EBAF0E94271CA031E7E2CD
:10231200BE07E0E08E07E0E09E0748F00E94271C1F
:10232200E0E1F7E260E070E00E94D320ECAF0E94AF
:10233200271CA83EE3E0BE07E0E08E07E0E09E0730
:1023420038F00E94271C0E94991D0E94D320EDAFF5
:102352000E94271CA436E0E0BE07E0E08E07E0E022
:102362009E0738F00E94271C0E9453200E94D3200F
:10237200EEAF0E94271C0E942C2028F00E94DE2033
:102382000E94D320EFAFFE01F1963F96FF93EF93A9
:102392000E94DE200E947625AF91BF91EC932330FC
:1023A20009F06CC00E945E200E94CB20E75F0E9471
:1023B2008420E7E7EAAFE4E7EBAFA0916003AA234A
:1023C20052F4E0915F03F09160030E946224E09373
:1023D2005F03F09360030E94F11F0E94B31B7723F7
:1023E20012F4E0E4EFAF0E94F11F0E94B31B0E94BF
:1023F200E42010F4E0E4EEAF0E94F11F0E94B31B50
:102402000E94ED2010F4E0E4EDAF0E94F11F0E9463
:10241200B31B0E94F62010F4E0E4ECAF0E94FF2010
:10242200A031E7E2BE072CF00E94FF200E940421A7
:10243200ECAF0E94FF20A83EE3E0BE072CF00E9412
:10244200FF200E940921EDAF0E94FF20A436E0E0A8
:10245200BE072CF00E94FF200E940E21EEAF0E94C8
:10246200FF201A972CF00E94FF200E941321EFAF49
:102472000E9418210E94FF200E941D21243009F091
:1024820064C00E945E200E94CB20E7570E948420F5
:10249200EEE3EAAFE4E7EBAFA0916203AA2352F4C2
:1024A200E0916103F09162030E946224E093610370
:1024B200F09362030E942421772312F4E0E4EFAF49
:1024C2000E9424210E94E42010F4E0E4EEAF0E9476
:1024D20024210E94ED2010F4E0E4EDAF0E942421BB
:1024E2000E94F62010F4E0E4ECAF0E942721A03114
:1024F200E7E2BE072CF00E9427210E940421ECAFE4
:102502000E942721A83EE3E0BE072CF00E9427216B
:102512000E940921EDAF0E942721A436E0E0BE0708
:102522002CF00E9427210E940E21EEAF0E9427214B
:102532001A972CF00E9427210E941321EFAF0E94CC
:1025420018210E9427210E941D21253011F50E9489
:102552005E200E94CB20E7570E948420EEE3EAAF80
:10256200E4E7EBAFE0E5ECAFA0912403A43620F062
:10257200B0E00E940E21EEAFA09124030E94D41F6E
:102582000E9445200E94A520A0912403BB270E94FF
:102592001D21263049F50E945E200E94CB20E7577C
:1025A2000E948420E0E0EAAFE5E0EBAFE8E7ECAFC1
:1025B200A881B981A83EE3E0BE071CF00E94092170
:1025C200EDAFA881B981A436E0E0BE071CF00E94FD
:1025D2000E21EEAFA881B9810E9413210E94A5208D
:1025E200A881B9810E941D21273009F04EC00E94A6
:1025F2005E200E94CB20E75F0E948420113030F1E0
:10260200ECE0EAAFA12F0E941420E436A0E0FA0722
:102612004CF0A12FB0E0E8ECF0E00E9436250E94D9
:102622004520EBAFA12F0E9414203A974CF0A12F26
:10263200B0E0E4E1F0E00E9436250E944520ECAFD4
:10264200A12F0E9414200E9445201EC0EBE0EAAF99
:102652000E942C21E436A0E0FA0738F0AB81BC815D
:10266200E8ECF0E00E943121EBAF0E942C213A9776
:1026720038F0AB81BC81E4E1F0E00E943121ECAFA3
:102682000E942C210E949F20EDAF283009F079C0D2
:102692000E945E200E947520E75D0E948420A09126
:1026A2005B03B0915C03A135EBEFBE0734F4E1E5C7
:1026B200FBEFE0935B03F0935C03A0915B03B091AB
:1026C2005C03A03BE4E0BE0734F0EFEAF4E0E09301
:1026D2005B03F0935C03A0915C03AA234AF4E0E459
:1026E200EDAFE0915B03F0915C030E94622404C0B1
:1026F200E0915B03F0915C03E0935D03F0935E0372
:10270200A0915D03B0915E03ECE3F0E00E943625F8
:10271200E0934103F09342030E943421ECE30E94D0
:102722001325A0915D03B0915E03AE1BBF0BA09376
:102732004303B093440324FE1BC00E9434211A9722
:1027420010F0E2E0E9AF0E9434210E943921EAAFA1
:10275200A0914303B09144030E94E31F0E949F2073
:10276200EBAFA0914303B09144030E943921ECAF37
:10277200E3E7EEAFE8E3EFAFE4E5DE01A05CBF4FD5
:10278200EC93293091F50E945E200E943E210E0EAC
:10279200A0E022FCA1E0EA2F0E9446210E0EA0E05A
:1027A20022FCA1E0EA2FE295E07FEE0FE00DEE8F32
:1027B200E9EAEF8F0E948E20A436E0E0BE0710F017
:1027C2000E9493200E948E200E94E31F0E949F205D
:1027D2000E94A5200E94AB2010F0E2E0E9AF0E9427
:1027E200B6200E9445200E94C120AC85A130C8F0CD
:1027F2000E941A20E9E7ECAFE0E5EDAFEEAFAC8561
:102802000E94D41F0E9445200E94A520AC85BB27B0
:102812000E941D210E944B210E94CB20E75F0E9453
:102822008420F29B07C00E944B210E943E21E00DB2
:10283200EF5FEE8F233609F0FCC351E0503130F4E4
:102842000E945921EAE0EC935F5FF8CFAA81EBE5A1
:102852000E946021EAE50E949824E02911F0E4E256
:10286200EA83AA81A53211F4ECE5EA83EA81E03039
:1028720029F4E0911003F0E0EF83F887AA81A130F8
:1028820029F4E0911103F0E0EF83F887AA81A230E6
:1028920029F4E0911203F0E0EF83F887AA81A330D4
:1028A20029F4E0911303F0E0EF83F887AA81A430C2
:1028B20029F4E0911503F0E0EF83F887AA81A530AF
:1028C20021F4EF89F0E0EF83F887AA81A63021F4A2
:1028D200E88DF0E0EF83F887AA81A73021F4E98D33
:1028E200F0E0EF83F887AA81A83029F4E09116037B
:1028F200F0E0EF83F887AA81A93019F4E0E0EF83D2
:10290200E887AA81AA3019F4E0E0EF83E887AA8178
:10291200AB3019F4E0E0EF83E887AA81AC3021F410
:10292200E4E2F0E0EF83F887AA81AD3021F40E945F
:10293200CA1CEF83F887AA81AE3021F4EB89F0E05C
:10294200EF83F887AA81AF3021F4EC89F0E0EF83BE
:10295200F887AA81A03121F4ED89F0E0EF83F887AE
:10296200AA81A13121F4EF85F0E0EF83F887AA81F3
:10297200A23121F4E889F0E0EF83F887AA81A3313C
:1029820021F4E989F0E0EF83F887AA81A43121F4E8
:102992000E94541CEF83F887AA81A53121F4ED81AE
:1029A200FE81EF83F887AA81A63129F4E091200302
:1029B200F0E0EF83F887AA81A73129F4E09122039E
:1029C200F0E0EF83F887AA81A83129F4E09121038E
:1029D200F0E0EF83F887AA81A93121F4E32FF0E038
:1029E200EF83F887AA81AA3121F40E94B11FEF83F5
:1029F200F887AA81AB3121F40E94B61FEF83F887D2
:102A0200AA81AC3131F4E0E023FCE1E0F0E0EF83B5
:102A1200F887AA81AD3121F40E944A1BEF83F8871F
:102A2200AA81AE3121F40E94561BEF83F887AA8156
:102A3200AF3129F4E0910803F0E0EF83F887AA812F
:102A4200A03229F4E0910A03F0E0EF83F887AA812B
:102A5200A13229F4E0910B03F0E0EF83F887AA8119
:102A6200A23229F4E0910C03F0E0EF83F887AA8107
:102A7200A33229F4E0910D03F0E0EF83F887AA81F5
:102A8200A43229F4E0910E03F0E0EF83F887AA81E3
:102A9200AC3529F4E0910703F0E0EF83F887AA81CF
:102AA200AD3521F4EC8DF0E0EF83F887AA81AE35E5
:102AB20021F4E985FA85EF83F887AA81AF3521F4FD
:102AC200EB8DF0E0EF83F887AA81A03621F4EA8D3E
:102AD200F0E0EF83F887AA81A13629F4E0911B0385
:102AE200F0E0EF83F887AA81A23629F4E091180377
:102AF200F0E0EF83F887AA81A33629F4E091170367
:102B0200F0E0EF83F887AA81E0E00E946021E3E031
:102B12000E946521E1E10E946521E2E10E946521B6
:102B2200E3E10E946521E5E10E946521EBE10E945B
:102B32006521EDE10E949824E02911F0F69A01C086
:102B4200F698A0E0F699A1E0EA2FE795E0E0E79594
:102B5200EF8FE0E0EE8FED8FE0930203AA81B0E009
:102B6200A7FDBFEF0E941321ECABAA81B0E0A7FD45
:102B7200BFEFEAE0F0E00E946825EDABAF81B885D7
:102B8200A031E7E2BE0728F0E0E1F7E20E9431213E
:102B9200ECAFAF81B885A83EE3E0BE0728F0E8EECF
:102BA200F3E00E943121EDAFAF81B885A436E0E0B9
:102BB200BE0718F00E946A21EEAFAF81B8851A975E
:102BC20028F00E946D210E949F20EFAF0E941821E1
:102BD200AF81B8850E943921DB01EC93EA81E030B4
:102BE20061F4EDE6EEABE9E7EFABE8E7E8AFEDE67F
:102BF200EBAFE4E5ECAFE0E5EDAFAA81E1E10E94E5
:102C02006021E2E10E946521E3E10E946521E5E1A4
:102C12000E946521EDE10E949824E02929F00E949A
:102C22006D210E949F20EFAFE7EAE0937A00A7E0D0
:102C32000E94B51C0E94D61CE7E2E0937A00AA81AA
:102C42000E94F61CAA81EEE00E946521E1E10E9449
:102C52009824E02911F0E1E06E2EAA810E94FB1C6B
:102C6200AA81EFE00E946521E2E10E949824E02916
:102C720011F0E2E06E2EAA81E7E00E946021E0E11D
:102C82000E9465210E94702111F0E3E06E2E0E94E5
:102C9200DB1CD39708F457C00E94101D0E94151D1B
:102CA200E62D0E941C1D20F0E8ECF0E00E94D61CEC
:102CB200E62D0E942C1D0E947521AC91A13008F4D2
:102CC20041C00E947C210E944C1D0E9410264CF49F
:102CD2000E9475210E9485210E9458240E94902101
:102CE20023C00E9499210E946E1DEF930E94992198
:102CF2000E94771DAF91EA2379F00E9475210E940C
:102D020085210E945D24A0936903B0936A03809396
:102D12006B0390936C0308C00E9499210E94801D4E
:102D22001CF00E949B210EC0A0916903B0916A031E
:102D320080916B0390916C030E94991D0E94602503
:102D42000E94D61C04C00E949E1D0E949B21AA8143
:102D5200AD3061F40E94A3210E9453200E943A20C8
:102D62000E94AC210E94B321E0E2ED8FAA81A5313D
:102D720061F40E94A3210E9453200E943A200E94E3
:102D8200AC210E94B321E0E6ED8FAA810E94F61CDD
:102D9200AA81EEE00E946521E1E10E949824E029E7
:102DA200A9F00E94BD21E4E00E94C12118F00E9416
:102DB200C721EEAB0E94DB1C1A9728F00E94C921A2
:102DC2000E949F20EFAB0E94CB21E8AFAA810E9414
:102DD200FB1CAA81EFE00E946521E2E10E94982497
:102DE200E029A9F00E94BD21E2E00E94C12118F071
:102DF2000E94C721EEAB0E94DB1C1A9728F00E94AA
:102E0200C9210E949F20EFAB0E94CB21E8AFAA818B
:102E1200E7E00E946021E0E10E9465210E947021AA
:102E2200A9F00E94BD21E1E00E94C12118F00E9498
:102E3200C721EEAB0E94DB1C1A9728F00E94C92121
:102E42000E949F20EFAB0E94CB21E8AFAA81A43160
:102E520089F40E94CD210E946A21EEAB0E94CD210D
:102E62000E94E31F0E949F20EFAB0E94CD210E948F
:102E72003921E8AFAA81A63121F40E94D221EBE0E8
:102E8200EDAFAA81A73121F40E94D221E0E4EDAF97
:102E9200AA81A83121F40E94D221ECE0EDAFAA81EF
:102EA200A93161F4A09125030E94D41F0E944520FC
:102EB200EEAB0E944B20EFABE7E7E8AFAA81AA3165
:102EC20089F40E94D9210E946A21EEAB0E94D92185
:102ED2000E94E31F0E949F20EFAB0E94D9210E9413
:102EE2003921E8AFAA81AB3159F4ECE7EAAFE7E761
:102EF200EBAFE8E7ECAF0E946D210E949F20EFAF9D
:102F0200AA81EDE10E946021EEE10E949824E0296D
:102F1200D9F0E3E7EAAFE8E3EBAFAA81AD3111F410
:102F2200EEE501C0E8E7ECAF0E94DE211A9738F027
:102F32000E94DE210E94E31F0E949F20EFAB0E94AD
:102F4200DE210E943921E8AFAA810E94F61CAA81E3
:102F5200E6E00E946521E7E00E949824E02911F052
:102F6200E3E7EAAFAA81EEE00E946021EFE00E946F
:102F72006521E0E10E949824E02931F0EDE6EAAF14
:102F8200E9E7EBAFE4E5ECAFAA81E1E10E94602161
:102F9200E2E10E9465210E94702111F0E8E7EBAFA7
:102FA200AA81AD3561F5E7E7EDAFEEE5EEAFE9E316
:102FB200EFAFFE01F1963F96AC8DA083E7EAE09376
:102FC2007A000E94B51C7E2EE7E2E0937A00E3E6E7
:102FD200E71528F4A72DB0E00E940E21EEABE9E040
:102FE200E71530F4A72D0E94D41F0E944520EFABB5
:102FF200A72DBB27EAE0F0E00E946825E8AFAA818E
:10300200AE3521F4EEE5EAAFE1E0EBAFAA81AF35F0
:1030120021F4EEE5EAAFE2E0EBAFAA81A03621F4BB
:10302200EEE5EAAFE3E0EBAFAA81A23611F4E0E10C
:10303200ED8F51E0503108F077C00E945921EC9198
:10304200E03021F40E945921EFE3EC930E945921D0
:10305200AC91A63021F40E945921EDE7EC930E9435
:103062005921AC91A13021F40E945921E6E0EC9360
:103072000E945921AC91A23021F40E945921EBE522
:10308200EC930E945921AC91A33021F40E94592162
:10309200EFE4EC930E945921AC91A43021F40E94F8
:1030A2005921E6E6EC930E945921AC91A53021F416
:1030B2000E945921EDE6EC930E945921AC91A73070
:1030C20021F40E945921E7E0EC930E945921AC912E
:1030D200A83021F40E945921EFE7EC930E94592174
:1030E200AC91A93021F40E945921EFE6EC930E94A1
:1030F2005921AC91AA3021F40E945921E0E0EC93CD
:103102000E945921AC91AB3021F40E945921E1E097
:10311200EC930E945921AC91AC3021F40E945921C8
:10312200E8E0EC935F5F86CFE0910203E695E695D7
:103132000E94E321EEA90E94E921EEA90E94F12159
:10314200EEA90E94FC21EEA90E940322EEA90E9490
:103152000A22EEA90E941122EEA90E941822E9A3D6
:10316200E0910203E695E695E6950E94E321EFA938
:103172000E94E921EFA90E94F121EFA90E94FC21FE
:10318200E8AD0E940322E8AD0E940A22E8AD0E9447
:103192001122E8AD0E941822EAA3E0910203E6950B
:1031A2000E94E321E8AD0E94E921E8AD0E94F121ED
:1031B200E8AD0E94FC21EFA90E940322EFA90E9420
:1031C2000A22EFA90E941122EFA90E941822EBA362
:1031D200E9AD0E94E321EAAD0E94E921EAAD0E9435
:1031E200F121EAAD0E94FC21EF8D0E940322EF8DB6
:1031F2000E940A22EF8D0E941122E0910203E170E7
:10320200EA2BECA3EEAD0E94E321EEAD0E941E225A
:10321200EEAD0E942422EEAD0E942D220E943722A2
:10322200EEAD0E943B22EEAD0E944422EEADE2954D
:10323200E170EA2BEDA3EDAD0E94E321EDAD0E941A
:103242001E22EDAD0E942422EDAD0E942D22E295B8
:103252000E940322EFAD0E943B22EFAD0E94442266
:10326200EFADE295E170EA2BEEA3EF8D0E944D22C5
:10327200EDAD0E94E921EDAD0E94F121EDAD0E947C
:10328200FC21ECAD0E940322ECAD0E940A22ECADBF
:103292000E941122ECAD0E941822EFA3EFAD0E9412
:1032A200E321EFAD0E941E22EFAD0E942422EFAD7A
:1032B2000E942D220E9451220E940322ECAD0E9404
:1032C2003B22ECAD0E944422ECADE295E170EA2B88
:1032D200E8A7EBAD0E94E321EBAD0E941E22EBAD0D
:1032E2000E942422EBAD0E942D22EE1FE0E0EE1F91
:1032F2000E9403220E9456220E943B220E945622D2
:103302000E9444220E945622E295E170EA2BE9A72C
:10331200EE8DE2950E94E321EBAD0E94E921EBAD37
:103322000E94F121EBAD0E94FC21EAAD0E94032232
:10333200EAAD0E940A22EAAD0E941122EAAD0E9481
:103342001822EAA70E9456220E94E3210E945622D6
:103352000E941E220E9456220E9424220E9456226D
:10336200E695E695E6950E945B22EAA9EE1FE0E06B
:10337200EE1F0E940322EAA9E2950E946122EAA9B5
:103382000E944422EAA9E295EF70E695E170EA2BE9
:10339200EBA7EAA9E695E695E6950E94E321EAA95C
:1033A200E695E6950E946722EAA90E946C22EAA9A4
:1033B2000E945B22EE8D0E943722EE8D0E947422C3
:1033C200EE8D0E947722EE8DE695E170EA2BECA756
:1033D200EE8D0E944D22EBA9E2950E946722EBA995
:1033E2000E94F121EBA90E947C22EBA90E943722C4
:1033F200EBA90E947422EBA9E6950E947722EBA921
:10340200E170EA2BEDA7EE8D0E9451220E94E3218A
:10341200ED8D0E946722ED8D0E946C22ED8DE69566
:10342200E6950E945B22E0910203E2950E9403224C
:10343200EE8DEE1FE0E0EE1F0E946122ED8DE6951B
:10344200E695E6950E947722ED8DE295E170EA2BF2
:10345200EEA7ED8D0E944D22ECA9E2950E94672213
:10346200ECA90E94F121ECA90E947C22EDA90E9404
:103472003722EDA90E947422EDA9E6950E947722D7
:10348200EDA9E170EA2BEFA7ED8D0E9451220E9477
:10349200E321EDA9E2950E946722EDA90E94F121A4
:1034A200EDA90E947C22ECA90E943722ECA90E947D
:1034B2007422ECA9E6950E947722ECA9E170EA2B2E
:1034C200E8AB33FE0DC051E0513150F4E52FF0E08E
:1034D200DE019096AE0FBF1FEFEFEC935F5FF4CF6C
:1034E2000E9480225D3078F40E948622A2E5B8E034
:1034F2000E947624E17011F45D9801C05D9A0E94E9
:103502008D225F5FEFCF0E9495225D3078F40E949A
:103512008622A0E3B8E00E947624E17011F45D985F
:1035220001C05D9A0E948D225F5FEFCF0E949522BB
:103532005D3078F40E948622A2E0B8E00E947624F0
:10354200E17011F45D9801C05D9A0E948D225F5F67
:10355200EFCF0E9495225D3078F40E948622A6E089
:10356200B8E00E947624E17011F45D9801C05D9A82
:103572000E948D225F5FEFCF0E9495225A3098F40D
:103582005E9885E28A95F1F7E9E0E51BA0E4B1E0F7
:103592000E947624E17011F45D9801C05D9A0E9448
:1035A2008D225F5FEBCF41E04131E8F451E05930C9
:1035B200C0F45E9885E28A95F1F7E42FF0E0DE012F
:1035C2009096AE0FBF1FAC91E8E0E51B0E946E24FF
:1035D200E17011F45D9801C05D9A0E948D225F5FD7
:1035E200E6CF4F5FE1CF5D9A85E28A95F1F7289A9F
:1035F2008DEC9AE00197F1F70E94A41DA82DEAE054
:103602000E94B1240E2AAA2DEAE00E94B1240E2AB9
:10361200AD2DEAE00E94B124E02929F0E0E0E09338
:103622004903E0934A03AB2DE4E60E94B6240E2E32
:10363200A0E0F099A1E00E94C01D39F0A4E6B0E03C
:103642000E949F22F09AE89433F80C94ED04EF96CE
:103652002296FFCFAA93E091C000E072E1F3E881E5
:10366200E093C60021960895A0913103B0913203F0
:103672000895A0918103B091820380918303909178
:1036820084030895E0E0F0E061EE75E40E94E72330
:103692000895E0913D03F0913E0308956627772750
:1036A2000E940F230E94AF250895E0914B03F091F1
:1036B2004C030895A0918903B0918A0380918B03F2
:1036C20090918C030895E0E0F0E060E271E40895E7
:1036D200A0913D03B0913E030895E0E0F0E00E9426
:1036E200CD240895A0914B03B0914C030895E0912D
:1036F200B103F091B2036091B3037091B4030895E2
:103702000E94D622ED93FC930895A0919D03B0915F
:103712009E0380919F039091A00308950E94992394
:10372200DF01CB01AFCFA0919903B0919A038091B1
:103732009B0390919C030895A0913F03B091400395
:103742000895E4E60E941325DF01E0919903F091C8
:103752009A0360919B0370919C03882799270E948A
:10376200B62508950E94B9250E94422308950E9419
:10377200D822ED93FC930895E0917103F0917203C6
:10378200609173037091740308950E941325DF0101
:10379200E091B903F091BA036091BB037091BC034D
:1037A200882799270E94B625DDCFE091A503F091E5
:1037B200A6036091A7037091A8030895E091A10365
:1037C200F091A2036091A3037091A4030895A091C4
:1037D2008503B091860380918703909188030895B1
:1037E200E0938503F09386036093870370938803C5
:1037F2000895A0918D03B0918E0380918F039091D3
:1038020090030895E0918503F09186036091870308
:10381200709188030895A0919503B09196038091C9
:103822009703909198030895E0915103F091520308
:1038320060915303709154030895E0935103F09300
:10384200520360935303709354030895A09151035C
:10385200B091520380915303909154030895E0E094
:10386200F0E060E070E00895E0E00E94B6240E2EE1
:103872000895A0916D03B0916E0380916F039091B2
:10388200700308950E22A0911C03ECE30E94B12460
:103892000895A0914903B0914A030895A091470366
:1038A200B09148031ACFE0914703F091480308957D
:1038B200A4E1B0E00E949F22E7EAE0937A00089533
:1038C200A4E00E943003EF2FF0E09E2EE7E2E093A7
:1038D2007A00E7EAE0937A000895A3E00E943003B9
:1038E200EF2FF0E08E2EE7E2E0937A00E7EAE09332
:1038F2007A000895A1E00E943003EF2FF0E0AE2E8F
:10390200E7E2E0937A000895EBE0E093C203E8EB8C
:10391200E093C3030895E8ECF0E0E0935703F093DB
:1039220058030895E0EDF7E0E0935903F0935A034A
:103932000895E0933503F093360308950E948E2490
:103942000E940F230E94AF250895E0933B03F0935A
:103952003C030895E0933F03F09340030895E093FE
:103962004703F093480308950E943003EF2FF0E0DD
:1039720008950E9430030E9483240E947F240895A8
:10398200E0937103F0937203609373037093740373
:103992000895E0913503F09136030895E7E2E0934C
:1039A2007A00E7EAE0937A000895E0932D03F0931A
:1039B2002E030895A0912D03B0912E030895FADFEE
:1039C200EAEFF0E00895F6DFEEE1F0E00E94C724AE
:1039D20008950E2EA52DE1E00E94B6240E22AC859C
:1039E200E5E00E94B124E0210895E5E00E949824D8
:1039F2000E2E0895E6E00E9498240E2E0895AD2D15
:103A0200EAE00E94B1240E2E0895A0E0F3FCA1E0AA
:103A1200E0E00E9498240E22A22FE3E60895E091AE
:103A22002D03F0912E030895F297ADE7B0E00E94C6
:103A3200EB240F010895F0E0DE015296AE0FBF1F96
:103A4200EC91F0E0D0010E942325AFDFB3DFA93C67
:103A5200E0E0BE070895F0E0DE015696AE0FBF1F0C
:103A6200EC91F0E0A7DF0E94EB24DF01E4E6F0E056
:103A72000E9423259ACFE02FF0E0DE011E96AE0FC2
:103A8200BF1F0895A0916503B091660380916703FB
:103A9200909168030895E8EEF3E060E070E00E9420
:103AA2006025DF01CB01BBDF662777270895EC9104
:103AB200F0E00E948E24A8E0BCE481E090E00E9445
:103AC2006025E0CFE0936503F0936603609367039C
:103AD200709368030895D6DFDECF0E945D24E5E08F
:103AE200F0E060E070E00E94E32408950E945D240B
:103AF200E4E1F0E060E070E00E94DB2408950E94BF
:103B02005D24A431E0E0BE07E0E08E07E0E09E071E
:103B12000895E0916D03F0916E0360916F037091CF
:103B22007003A0E5B4E180E090E00E941E25CACFB8
:103B3200E8EEF3E060E070E00895E0E0E0932D034A
:103B4200E0932E030895A92DEAE00E94B1240E2EDF
:103B52000895A22FE3E60E94B1240895A0E0F0FCAC
:103B6200A1E0E0E00E9498240895A09123037CCE76
:103B7200E09122037EDEFF27662777270895E0E0A3
:103B82000E949824E0210895ED81FE81A0917103A5
:103B9200B091720380917303909174036627772723
:103BA2000E94DB240E2EEAE0F0E060E070E00E946A
:103BB200E3240895E0935703F09358030895DCDD5E
:103BC200AD81BE81882799270E945D240895A63081
:103BD200E0E0BE07E0E08E07E0E09E070895A091D6
:103BE2005703B09158030895E0915703F091580399
:103BF2000895ED81FE81A0917103B09172038091CD
:103C0200730390917403662777270895E32FA09199
:103C1200AD03B091AE038091AF039091B003FF2743
:103C2200662777270E940F230895C4DEEAE00E94E8
:103C320013250895E32FF0E0A091AD03B091AE03F8
:103C42008091AF039091B0030E948E240E940F23B3
:103C520089CD662777270E940F230E949923089512
:103C6200A0915903B0915A0308950E9493240E948F
:103C7200B62578CDA32FBB27E091AD03F091AE031B
:103C82006091AF037091B003F0CFE0915903F091CE
:103C92005A030895EAE0F0E00E94362586CEE091CC
:103CA2001203E7DDFF27662777270895E093630372
:103CB200F09364030895E0911203F0E0DADD0E94CC
:103CC2008E240E945D2408950E941925A091630309
:103CD200B09164030895E0916303F0916403089541
:103CE200A0911203BB27E0916D03F0916E036091E6
:103CF2006F03709170030E9493240E945D240895C3
:103D02000E2EA0911C03ECE30E94B1240E22089512
:103D1200E0911103A0E0B0E00E94EA25E0911203D5
:103D2200A1E0B0E00E94EA25E0911303A2E0B0E036
:103D32000E94EA25E0911503A3E0B0E00E94EA2583
:103D4200EF89A4E0B0E00E94EA25E88DA5E0B0E0AA
:103D52000E94EA25E98DA6E0B0E00E94EA25E09102
:103D62001603A7E0B0E00E94EA25E0911703A8E05D
:103D7200B0E00E94EA25E0911803A9E0B0E00E94B9
:103D8200EA25E0911B03AAE0B0E00E94EA2501DEE9
:103D9200AEE1B0E00E94E225EB89A4E1B0E00E942E
:103DA200EA25EC89A5E1B0E00E94EA25ED89A6E1C9
:103DB200B0E00E94EA25EF85ABE0B0E00E94EA2580
:103DC200E889ACE0B0E008950E94EA25E989ADE017
:103DD200B0E00E94EA25ED81FE81A2E2B0E00E94FD
:103DE200E225E0912003AEE0B0E00E94EA25E091F6
:103DF2002203AFE0B0E00E94EA25E0912103A0E1B6
:103E0200B0E00E94EA25E32FA1E1B0E00E94EA259A
:103E1200E985FA85A4E2B0E00E94E225EB8DA2E1F9
:103E2200B0E00E94EA25EA8DA3E1B0E00E94EA2513
:103E3200E0919903F0919A0360919B0370919C0326
:103E4200A6E2B0E00E94D8220E94E225E0913B0364
:103E5200F0913C03A8E2B0E00E94E225E0913F032A
:103E6200F0914003ACE2B0E00E94E225E0E023FCE6
:103E7200E1E0A7E1B0E00E94EA2515DDAAE2B0E0A8
:103E82000E94E225E0910803A8E1B0E00E94EA2541
:103E9200E0910A03A9E1B0E008950E94EA25E091C9
:103EA2000B03AAE1B0E00E94EA25E0910C03ABE12A
:103EB200B0E00E94EA25E0910D03ACE1B0E00E947F
:103EC200EA25E0910E03ADE1B0E00E94EA250895F3
:103ED200EAE00E94B6240E2E0895AA2DEAE00E947E
:103EE200B1240E2EA0E027FCA1E0E0E00E9498247D
:103EF2000E220895A0E0F2FCA1E0E0E00E949824E6
:103F02000E220895A82DEAE00E94B1240E2E0895F3
:103F1200E0E00E9498240E220895E0910F03F0E061
:103F2200E65FFC4F08950E22A22FE3E60E9498243A
:103F3200E0210895A22FE3E60E949824E02108954B
:103F4200E0912A03EF5FE0932A03E0912903A09115
:103F52002A03EA170895A0913B03B0913C03089508
:103F6200E0913B03F0913C030895E0913F03F0910F
:103F720040030895E091AD03F091AE036091AF0369
:103F82007091B0030895A0E0B0E080E09FE30E944A
:103F920049230895E0939D03F0939E0360939F034A
:103FA2007093A0030895B0E0EAE0F0E00E943625A5
:103FB2000895E0917D03F0917E0360917F037091FB
:103FC20080030895EAE0F0E00E9423250895A0917D
:103FD2007D03B0917E0380917F03909180030895C9
:103FE200ABDBAFCBE0937903F0937A0360937B036F
:103FF20070937C030895F0E0EA0FFB1FE09339030E
:10400200F0933A03AEE30C942B1B0E942B1BA0E00F
:104012000C942B1BE0913A03AE2F0E942B1BA09114
:1040220039030C942B1BB0E0E2E0F0E00E9436254D
:104032000895EAE0E9AFEAAFEBAF0895A091750306
:10404200B0917603809177039091780308950E944E
:10405200E3240E2EF3CFAA30E0E0BE07E0E08E07A5
:10406200E0E09E07089505DCEAE0F0E060E070E041
:1040720008950E946025DF01CB01EAE0F0E060E0F4
:1040820070E00E947A250895DF01EAE0F0E00E94E4
:1040920068250895A0912503BB27EAE0F0E00E947D
:1040A20068250895E4E6F0E060E070E00895C6DF78
:1040B200EAE0F0E060E070E00895E0912603E1704C
:1040C200EE0FE058AE2FE0912603E695E695E170FB
:1040D200EE0FEE0FEA0F0E2EA0E0F199A1E0EA2F0B
:1040E200EE0FEE0FEE0F08950E0EA0E020FCA1E001
:1040F200EA2FE295E07FE00DEE8FA0E022FCA1E046
:10410200EA2FEE0F08950E2EA0E022FCA1E0EA2F86
:10411200EE0FEE0FE00DEF8F0895A0913303B091F3
:1041220034030895FADFE4E6F0E00E942325DF017C
:10413200EAE0F0E00E946525EEAF0895DF01EAE0D3
:10414200F0E00E9465250895EFAFFE01F1963F96DB
:10415200BF010895E2DFEAE0F0E00E946525DB019D
:10416200EC93A0910103AA300895A0910103BB270B
:10417200EAE0F0E00E946825EAAFA091000313CFC5
:10418200EBAFA0910003BB27EAE0F0E00E946825B4
:10419200ECAF0895E00DEE8FA0E022FCA1E0EA2F43
:1041A200EE0F08950E943B25DF01CB01EAE0F0E02B
:1041B20060E070E00E947625089548DBEAE0F0E0D6
:1041C20060E070E00895DF01CB01E0E0F0E060E143
:1041D20071EC0E942C240895DF01CB01E0E0F0E0B5
:1041E20066EC72EC0E942C240895DF01CB01E0E022
:1041F200F0EC69E774EC0E942C240895A0915F030F
:10420200B09160030895E0E1F7E20E9436253CCFC9
:10421200E8EEF3E00E94362537CFE4E6F0E00E94B4
:10422200362532CFEAE0F0E00E9436252DCFFE019E
:10423200F1963F96BF010895EAE0F0E00E946825FA
:10424200DB01EC93089578DAE4E69FCAA09161035A
:10425200B09162030895EB81FC81F695E79508958C
:104262000E9423256BCFA0914103B0914203089590
:10427200EAE0F0E00E94652508950E0EA0E020FC21
:10428200A1E0EA2FE295E07F0895E295E07FEE0F4C
:10429200EE0F0895E0912603E170EE0FE0580E2E26
:1042A200A0E0F199A1E0EA2FEE0FEE0FEE0F0895D4
:1042B200E52FF0E0DE01D196AE0FBF1F08950E94F8
:1042C20098240E2EAA8108950E9498240E2AAA816B
:1042D2000895E4E6F0E0C4CFAF81B88573CEE3E1A0
:1042E2000E949824E0290895E62DF0E0DE011E9652
:1042F200AE0FBF1F0895A0916903B0916A03809128
:104302006B0390916C030895EC91F0E00E948E246F
:10431200A8E0BCE481E090E00E946025ECCFE0934D
:104322006903F0936A0360936B0370936C030895BF
:10433200E2DFB1CBE985FA859CDA662777270E940E
:104342001E25EDCFA0917103B0917203809173038A
:10435200909174030895EEABF5DFEAE0F0E060E0DF
:1043620070E087CEEFABEEDFEAE0F0E060E070E015
:104372000E947A25E8AF089552DBF695E79515CBB2
:10438200ED8F18DBA436E0E0BE07089513DBA1CF62
:1043920011DB18CE0FDB6CCFA0914F03B09150030D
:1043A2000895E9E3EAAFE0E5EBAFEEE3ECAF0895A1
:1043B200A0913703B09138030895A0914503B091BD
:1043C20046030895E170E795E0E0E795AE2F089582
:1043D200E295EF70E695E17058DFEA2BAE2F089573
:1043E200E295EF70E695E695E170E295E07FEE0FDB
:1043F200EA2BAE2F0895E295E170E295E07FEA2B79
:10440200AE2F0895E170EE0FEE0FEE0FEA2BAE2FF6
:104412000895E695E170EE0FEE0FEA2BAE2F0895A8
:10442200E695E695E170EE0FEA2BAE2F0895E6953C
:10443200E695E695E170EA2B0895E695E17025DFB1
:10444200EA2BAE2F0895E695E695E170E295E07FBE
:10445200EE0FEA2BAE2F0895E695E695E695E1700C
:10446200E295E07FEA2BAE2FEF8D0895E695E69573
:10447200E695C8CFE295EF70E695E170EE0FEE0F8C
:10448200EA2BAE2F0895E295EF70E695E695E1707E
:10449200EE0FEA2BAE2F0895E295EF70E69592CFDC
:1044A200E295EF70E695E6950895FE01E05CFF4F18
:1044B200E0810895E170E295E07FEA2BAE2F089546
:1044C200E170EE0FEE0FEA2BAE2F0895E170DDDE04
:1044D200EA2BAE2F0895E695E170E295E07FEE0FAC
:1044E200EA2BAE2F0895E695E695EACFE170EE0F3E
:1044F200EA2BAE2F0895E295EF70E695DBCF289870
:1045020085E28A95F1F751E008955E9885E28A95F1
:10451200F1F7ECE0E51B089585E28A95F1F75E9AE2
:1045220085E28A95F1F708955D9A85E28A95F1F719
:10453200289A84E191E00197F1F7E1CF109639F0E2
:104542008DEC9AE00197F1F7A8951197C9F70895B4
:10455200552342F4503811F4E0FF04C03196691F2C
:10456200791F6BF050E8572711F45F93CFC05F3F7C
:1045720031F0660F000C57956795752F08955F937C
:1045820000200AF0CFC0C8C050E8192E1522880FAB
:10459200991F9527550F879550E8072E0522660F1C
:1045A200771F7527550F67950895689401C0E894A1
:1045B2005F93F2DF703818F07F3F08F4A7C056E12E
:1045C200571BAAF4519558300EF4593030F0EFEFE2
:1045D200FFEF6FEF7FE777F91AC077275523B9F01E
:1045E200EE0FFF1F661F771F5A95D1F710C077276E
:1045F200583028F0EF2FF62F672F5850F9CF552358
:1046020031F076956795F795E7955A95D1F70020A1
:104612000AF45BD15F910895689401C0E8943097E1
:1046220060407040B1F0002426F0772312F4009429
:104632004CD1172E7EE1112032F07A95EE0FFF1F3A
:10464200661F111CF9CFEF2FF62F612D5F938ADFC2
:104652005F9108954F93AF01FD01DA01AB01BC01F7
:10466200CA01402D012C142E4F910895EA0FFB1F11
:10467200681F0895E095F0956095EF5FFF4F6F4FCB
:1046820008955F9381DF903871F150E8152604C0D8
:104692005F937ADF903839F1703821F1572F591B27
:1046A2002BF112F4D7DFFACF583118F0AA27BB2723
:1046B2008827583028F0AB2FB82F88275850F9CFC9
:1046C200552329F08695B795A7955A95D9F7502D78
:1046D200512572F0CBDF38F46795F795E79573951E
:1046E20013F420C0B7DF3EDF5F910895D8F7FBCF08
:1046F200EA1BFB0B680B51F010F40094BBDF66233E
:1047020092F3EE0FFF1F661F7A95CBF7EE27FF2776
:10471200662777275F910895EFEFFFEF6FE77FEF4F
:104722005F910895EFEFFFEF6FE77FE75F910895E5
:104732005F932ADF703851F3903841F301240894D3
:10474200791F23F41CF300203AF3ECCF0F921F934E
:104752002F933F934F93112722279927689FA001F8
:104762008F9F302D410D591F6B9F300D411D591FD9
:104772008E9F27D0BF9F25D06A9F23D0BE9F1DD07A
:10478200AF9F1BD0AE9F110D291F391F491F591F03
:10479200E32FF42F652F522F4F913F912F911F91AD
:1047A2000F9066232AF0550FEE1FFF1F661F02C0EF
:1047B20073954BF2CDDE5F910895100D211D391FC7
:1047C20002C0200D311D491F591F08955F93DCDE81
:1047D200703821F411200AF49FCFA4CF903809F445
:1047E20095CF01240894970B1BF4D4F30020F3CF48
:1047F200792F1F932F933F934F9311241127222731
:1048020033274427552790E2AE17BF078607410793
:1048120030F0AE1BBF0B860B410B089401C088948D
:10482200551F221F331F111CAA1FBB1F881F441FA5
:104832009A9551F7F901612D4F913F912F911F9157
:10484200662332F0550FEE1FFF1F661F7A9543F263
:104852007FDE5F91089599239AF0772342F09717AC
:1048620048F029F4AE17BF07860720F031F098947C
:1048720088940895989408940895189488940895B3
:104882007723C2F7971798F3A9F7EA17FB07680788
:1048920088F399F3ECCFDFDFE1E009F008F0EE27CF
:1048A2000895D9DFE1E009F008F4EE270895EA0F50
:1048B200FB1F681F791F0895AE1BBF0B860B970B5A
:1048C2000895F195E195F0400895F0956095709501
:1048D200E195FF4F6F4F7F4F0895EE230E2EEA2F83
:1048E20019F0E6950A94E9F70895EE230E2EFD01DC
:1048F20021F0F695E7950A94E1F70895F695E79584
:10490200F695E795F695E795F695E7950895FE2FC6
:10491200FF0FFF0B6F2F7F2F08956F2F660F660B10
:10492200762F08958B2F880F880B982F0895EA17FA
:10493200E1E009F0EE270895EA17E1E009F4EE2735
:104942000895AE17E1E00CF4EE270895AE17E1E00A
:104952000CF0EE270895EA17E1E00CF0EE27089537
:10496200AE17E1E008F0EE270895EA17E1E008F05B
:10497200EE270895EA17FB07E1E009F0EE27089514
:10498200AE17BF07E1E008F4EE270895AE17BF07A0
:10499200E1E008F0EE270895EA17FB07E1E008F0EE
:1049A200EE270895EA17FB0768077907E1E009F0A7
:1049B200EE270895AE17BF0786079707E1E00CF0D0
:1049C200EE270895EA17FB0768077907E1E00CF084
:1049D200EE270895FA9FF02DEB9FF00DEA9FE02D50
:1049E200F10D08957A9F702D6B9F700DF89F700DD9
:1049F200E99F700D6A9F602D710DFB9F600D711D07
:104A0200E89F600D711D8827FA9FF02D610D781FB8
:104A1200EB9FF00D611D781FEA9FE02DF10D681FDD
:104A2200781F08956E2F6A9FF0016B9FF00D089515
:104A320074D0D0DF0EF445DF08957DD0D3DF0EF4BD
:104A420044DF08950024112490E1AA0FBB1F001C2B
:104A5200111C0E1A1F0A18F40E0E1F1E01C0A160AF
:104A62009A9599F7FD01D001089557D0EBDF0EF426
:104A720028DF08953F934F935F9300241124442726
:104A8200552730E2AA0FBB1F881F991F001C111C5B
:104A9200441F551F0E1A1F0A460B570B28F40E0E01
:104AA2001F1E461F571F01C0A1603A9559F7FD010D
:104AB200BC01D001CA015F914F913F9108953BD053
:104AC200D9DF0EF402DF0895BDDFFD010895E894F9
:104AD200B7FF04C0A095B09511966894F7FDF1DE7A
:104AE200B1DFFD010EF4EDDE0895C4DFFD01BC016E
:104AF2000895E89497FF09C0A095B0958095909588
:104B0200AF5FBF4F8F4F9F4F689477FDDEDEB2DFFE
:104B1200FD01BC010EF4D9DE0895E894F7FF02C04E
:104B2200D0DE6894B7FF06C0A095B095119600F844
:104B3200039400FA0895E89477FF02C0C6DE6894F1
:104B420097FF0BC00024A095B09580959095119683
:104B5200801D901D00F8039400FA0895ED93FD93D3
:104B62006D937C930895689401C0E89401D057DD59
:104B7200182E862F612D192E972F712D1B2EBF2FC8
:104B8200F12D1A2EAE2FE12D0895129602D0BF01FB
:104B92001297119602D0FE2F1197F999FECFFF932B
:104BA200FFB7F894A1BDB2BDF89AE0B5FFBFFF917F
:104BB200089507D012960F01FB0103D0F00112975E
:104BC200089507D01196EF93EF2F03D0EF9111972D
:104BD2000895F99B02C0A895FCCF9FB7F894A1BD98
:104BE200B2BDF89A80B5E81719F0E0BDFA9AF99AC1
:104BF2009FBF089500240E160F06060607060895A5
:104C020000240A160B06089500240A160B0608064D
:104C120009060895EA17FB07680779070895AE1792
:104C2200BF07860797070895E894EE2309F0689472
:104C32000895AC0FBD1F05900D928A95E1F7089576
:00000001FF
